:0200000480007A
:1000000037F1FF7FEF00C018EF008006730000009B
:10001000938B0600130C0700938C0700130F01004D
:100020009303050013051000635C75001301018044
:10003000130305006B500300130515006FF0DFFE7E
:1000400013010F0013050000930F0600938D0300AA
:10005000EBE0BF01170500001305852A6B40050082
:1000600017030000130303FB6B000300678000000D
:10007000130101FF23261100232481001304010131
:10008000B707008193870700370700811307C76010
:10009000B70600819386C65C370600801306460DBE
:1000A0009305100013050001EF0000391300000054
:1000B000EF00402193070500E38C07FE9307000043
:1000C000138507008320C10003248100130101016F
:1000D00067800000130101FD232611022324810201
:1000E00013040103232EA4FC232CB4FCEF00804056
:1000F0002326A4FEEF0080422324A4FEEF008044C8
:100100002322A4FE032784FD8327C4FDB307F70041
:100110002320F4FE832704FE939727000327C4FEC1
:10012000B307F70083A60700832704FE93972700F1
:10013000032784FEB307F70003A70700832704FE05
:1001400093972700032644FEB307F6003387E600A3
:1001500023A0E700832784FD138717009307070078
:1001600093971700B387E70093973700B387E700AB
:100170009397270013850700EF0000281300000065
:100180008320C10203248102130101036780000060
:1001900097020001938202EB1303000093037000A7
:1001A00023A0620023A2620023A4620023A672009F
:1001B00023A862006780000097020001938282E812
:1001C00003A382001303130023A4620013834201DC
:1001D00083AE420093935E0033037300032E050049
:1001E0002320C301032E45002322C301032E8500D3
:1001F0002324C301032EC5002326C301032E0501BA
:100200002328C301032E4501232AC301032E8501A0
:10021000232CC301938E1E00130F20036394EE0161
:10022000930E000023A2D201678000009702000114
:10023000938242E103A382001303F3FF23A462002D
:100240001383420183AE0200930F2003138F0E002D
:10025000130F1F006314FF01130F000023A0E2011E
:1002600093935E0033037300032E03002320C50124
:10027000032E43002322C501032E83002324C5013E
:10028000032EC3002326C501032E03012328C50125
:10029000032E4301232AC501032E8301232CC5010C
:1002A00067800000970200019382C2D903A38200F5
:1002B00013050000130E200363146E0013051500D0
:1002C00067800000970200019382C2D703A38200D7
:1002D00013050000130E000063146E0013051500D3
:1002E00067800000970200019382C2D503A3C20079
:1002F00083A3020133B5630067800000130101FD91
:10030000232611022324810213040103EFF09FFB33
:10031000930705006384070073000000930744FD02
:1003200013850700EFF09FF08327C4FD13810700BA
:10033000032584FD832544FD032604FE832644FE15
:10034000032784FE8327C4FEEFF09FCC73000000D8
:10035000130000008320C102032481021301010362
:1003600067800000130101FD23261102232481026E
:1003700013040103930901006F000005B707008112
:100380009387070483A7070113871700B707008126
:100390009387070423A8E700930744FD138507000C
:1003A000EFF0DFE88327C4FD13810700032584FDF8
:1003B000832544FD032604FE832644FE032784FE92
:1003C0008327C4FEEFF0DFC9EFF0DFEF93070500EE
:1003D00063980700EFF01FF193070500E39007FA19
:1003E00013810900130000008320C102032481024D
:1003F0001301010367800000130101FD2326810220
:1004000013040103232EA4FC232604FE6F00000125
:100410008327C4FE938717002326F4FE0327C4FE18
:100420008327C4FDE346F7FE130000000324C10246
:100430001301010367800000130101FB232611044F
:1004400023248104130401052326A4FC2324B4FCE3
:100450002322C4FC2320D4FC232EE4FA232CF4FA18
:1004600013090100232604FE6F00C005B709FFFF32
:10047000330131018327C4FE2328F4FC832784FC45
:10048000232AF4FC93070100232CF4FC832744FC6B
:10049000232EF4FC832704FC2320F4FE8327C4FBD3
:1004A0002322F4FE832784FB2324F4FE930704FD18
:1004B00013850700EFF05FD08327C4FE93871700F2
:1004C0002326F4FE0327C4FE8327C4FCE360F7FA67
:1004D00013010900EFF01FE913054006EFF0DFF10B
:1004E000130000008320C1040324810413010105CB
:1004F00067800000130101FF23268100232471017E
:100500001304010193870B00138507000324C10026
:10051000832B81001301010167800000130101FF9B
:1005200023268100232481011304010193070C0079
:10053000138507000324C100032C8100130101016E
:1005400067800000130101FF23268100232491010D
:100550001304010193870C00138507000324C100D5
:0C056000832C8100130101016780000062
:02000004810079
:1005CC000100000001000000060000000000000017
:1005DC000300000001000000010000000200000008
:1005EC0000000000030000000600000007000000EF
:1005FC0005000000070000000700000009000000D3
:10060C0000000000020000000200000000000000DA
:10061C0005000000000000000100000001000000C7
:10062C0004000000020000000000000000000000B8
:10063C0003000000020000000300000002000000A4
:040000058000000077
:00000001FF
